:020000040000FA
:020000005F2D72
:08000800FF000308FE000A08D6
:10001000FC000408FD008312031300308A00233023
:100020008100A20A073022020318A2012114A30FA3
:100030001C28A40F1C28A1143E08003E03193528D3
:100040002F1C332885147A230130842300001E30AE
:10005000A500851007308423851406308423A50B62
:100060002928851057287A2337286F2368231830CA
:10007000A6003830FB00FA01220803196320013082
:10008000220203196F200230220203197B20033061
:10009000220203198720043022020319932005301D
:1000A000220203199F20063022020319AB2085018A
:1000B00087010B117D0884007C088A007E0883007C
:1000C000FF0E7F0E09007B21A60B63280E227B21E9
:1000D00014227B2122227B2173237B210800DD2136
:1000E000A60B6F280E22DD211422DD212222DD2124
:1000F0007323DD210800B720A60B7B280E22B72032
:100100001422B7202222B7207323B7200800E8204A
:10011000A60B87280E22E8201422E8202222E820BD
:100120007323E82008001921A60B93280E22192119
:1001300014221921222219217323192108004A218E
:10014000A60B9F280E224A2114224A2122224A214C
:1001500073234A210800AC21A60BAB280E22AC2148
:100160001422AC212222AC217323AC210800A6303A
:10017000840001080002031C7A14AC3084000108DA
:100180000002031CFA14AA30840001080002031CB8
:100190007A15AE30840001080002031CFA15B03055
:1001A000840001080002031C7A16B33084000108A1
:1001B0000002031CFA16831603137B0885007A08D5
:1001C0008700831203130430850000308700080085
:1001D000A830840001080002031C7B15C93084008C
:1001E00001080002031CFA14C73084000108000251
:1001F000031C7A15AF30840001080002031CFA15B5
:10020000A230840001080002031C7A16B230840078
:1002100001080002031CFA16831603137B088500ED
:100220007A088700831203130030850001308700AD
:100230000800C530840001080002031C7B15C33090
:10024000840001080002031C7A14C63084000108EF
:100250000002031C7A15BC30840001080002031C54
:10026000FA15BF30840001080002031C7A16C03062
:10027000840001080002031CFA16831603137B088E
:1002800085007A088700831203130030850002304E
:1002900087000800C430840001080002031C7B159D
:1002A000C230840001080002031C7A14C8308400A4
:1002B00001080002031CFA14A130840001080002A6
:1002C000031CFA15BE30840001080002031C7A16D4
:1002D000C130840001080002031CFA1683160313C0
:1002E0007B0885007A08870083120313003085009D
:1002F000043087000800A930840001080002031CB4
:100300007B15A730840001080002031C7A14AD306D
:10031000840001080002031CFA14AB3084000108B9
:100320000002031C7A15B130840001080002031C8E
:100330007A16A430840001080002031CFA16831602
:1003400003137B0885007A088700831203130030AB
:100350008500083087000800B630840001080002DC
:10036000031C7B15B430840001080002031C7A14BE
:10037000BA30840001080002031CFA14B83084006B
:1003800001080002031C7A15BD3084000108000238
:10039000031CFA15A530840001080002031CFA169C
:1003A000831603137B0885007A08870083120313E2
:1003B00000308500103087000800B7308400010845
:1003C0000002031C7B15B530840001080002031CE9
:1003D0007A14BB30840001080002031CFA14B930FF
:1003E000840001080002031C7A15A0308400010873
:1003F0000002031CFA15A330840001080002031C4C
:100400007A16831603137B0885007A088700831207
:100410000313003085002030870008000310270DEB
:10042000B0001B22B30008000310270D013EB000EE
:100430001B22B400080002308A003008263E031850
:100440008A0A820033088A00340882000234663443
:100450000234713402347934023481340234893400
:1004600002349134023499340234A5340234A9346C
:100470000234B5340234B9340234C5340234C934D8
:100480000234D5340234D9340234E5340234E93448
:100490000234F5340234F9340334053403340934B6
:1004A0000334153403341934033425340334293424
:1004B0000334353403343934033445340334493494
:1004C000033455340334593403346534AE013030C9
:1004D000B20029186E2A0630A700672B0130A7004A
:1004E000672B2918762A0030A700672B0230A70057
:1004F000672B29187E2A0030A700672B0330A7003E
:10050000672B2918862A0430A700672B0330A70021
:10051000672B29188E2A0030A700672B0530A7000B
:10052000672B2918962A0730A700672B0030A700F1
:10053000672B2918A32A003032070319A12AB20B0E
:10054000672B2E14672BA701672B2908AD00A70A7C
:10055000672B2D082906031DAF2AA701672B291831
:100560002C10291C2C14A70A672B2908AD00A70AF8
:10057000672B2D082906031DBF2AA701672B291801
:100580002B12291C2B16A70A672B2908AD00A70AD6
:10059000672B2D082906031DCF2AA701672B2918D1
:1005A000AB11291CAB15A70A672B2908AD00A70AB8
:1005B000672B2D082906031DDF2AA701672B2918A1
:1005C0002B11291C2B15A70A672B2908AD00A70A98
:1005D000672B2D082906031DEF2AA701672B291871
:1005E000AB10291CAB14A70A672B2908AD00A70A7A
:1005F000672B2D082906031DFF2AA701672B291841
:100600002B10291C2B14A70A672B2908AD00A70A59
:10061000672B2D082906031D0F2BA701672B29180F
:10062000AA12291CAA16A70A672B2908AD00A70A37
:10063000672B2D082906031D1F2BA701672B2918DF
:100640002A12291C2A16A70A672B2908AD00A70A17
:10065000672B2D082906031D2F2BA701672B2918AF
:10066000AA11291CAA15A70A672B2908AD00A70AF9
:10067000672B2D082906031D3F2BA701672B29187F
:100680002A11291C2A15A70A672B2908AD00A70AD9
:10069000672B2D082906031D4F2BA701672B29184F
:1006A000AA10291CAA14A70A672B2908AD00A70ABB
:1006B000672B2D082906031D5F2BA701672B29181F
:1006C0002A10291C2A14A70A672BA7013114080035
:1006D0002E10AE10851EAE14051E2E140800291013
:1006E00085192914080028082702031C792B2708DC
:1006F000A80008002F10BE030310BD0CBC0CBB0CDF
:10070000BA0C03182F140800B500B50B852B080090
:10071000BB01BC01BD01A030BA00B809381C3B14B4
:100720003818BB14361E3B15361ABB15B61D3B16C2
:10073000B619BB16361D3B173619BB17B61C3C1431
:10074000B618BC14361C3C153618BC15B71E3C1622
:10075000B71ABC16371E3C17371ABC17B71D3D1405
:10076000B719BD14371D3D153719BD15B71C3D16FA
:10077000B718BD16371C3D173718BD172130BE00FE
:100780000800BF000000BF0BC22B0800C70A4708C3
:10079000103C0319C7014708B900F9010800C70355
:1007A0004708013E031DD72B0F30C700B900F901E0
:1007B00008002A08C700B900F03E031CE32B0F30E5
:1007C000C7024708DC2BF9010800C0002110211CDA
:1007D000E72BC00BE62B0800470ACA00C901CB0172
:1007E000CC01CD01CE0138305818CD00FF30162590
:1007F000C901CA01CB010130162508000530C1002E
:10080000AC30C2000310470DF9008B139F258B17E6
:10081000C4000314470DF9008B139F258B17C200EA
:100820004408C100080021304102031D1B2C42086E
:10083000790744242D2C8B130A08C500410878073A
:10084000DC00031042087907DD000318DC0AA62546
:10085000C60045088A0046088B17F90F302CF80AA5
:100860000800831603139C18332C8B131C1579086E
:100870009B0077089A0055309D00AA309D009C147B
:100880008B178312031308008B13831603139C1812
:10089000472C1C119B009C131C141A088312031371
:1008A0008B170800DE304424D80008005224581C5E
:1008B0005B2C58105C2C5814DE30F9005808F700F7
:1008C0003124EC23EC230800FE23F901F801132462
:1008D000C800C8131324D700D70A1324D900311C29
:1008E0008D2C07302B02031D782CD923B101642CE9
:1008F000AB08031D8D2C20302A020319C62321309A
:100900002A020319CF2300302A020319C7010C3031
:100910002A0203195624B101642C2E0803199F2CB6
:10092000EC23EC232E18972CAE189B2C642CC6239A
:10093000EC23EC23922CCF23EC23EC23922C0F30CE
:1009400048020319CA241030480205308A000319EE
:10095000CC2504308A00113048020319E6241230F5
:10096000480208308A0003194B2004308A003E08F0
:10097000003E031DC72CA11CC72CA110581CC22C63
:10098000C623642C0730B6003908B7008823D90B7A
:100990006F2C642C1324C9001324CA001324CB0029
:1009A0001324CC001324CD001324CE00C0304905FD
:1009B000DA000310DA0CDA0CDA0CDA0CDA0CDA0CE6
:1009C000DA0A57081625DA0BE12C08001324C900AF
:1009D0001324CA001324CB001324CC001324CD000D
:1009E0001324CE001324CF001324D0001324D100ED
:1009F0001324D2001324D3001324D4001324DA00C8
:100A0000DA0AC91B082D57081625DA0B012D080034
:100A100007308A004E2705308A005708E5232E1834
:100A2000152D3118152DDA0B012D0800D600A03038
:100A300084005030DB008001840ADB0B1B2D063064
:100A40008A007B2605308A005608E523080002301C
:100A50002702031C0301C9000030CA00013016251B
:100A60002E080319432DA801A7013E08003E031DCF
:100A7000302D2E08CA00C90101301625B6010C30F0
:100A8000B7008823302D311C272DB101F030C9006B
:100A9000CA017F301625C901CA013F301625F03042
:100AA000C900CA017F3016252A08C9002B08CA00D0
:100AB000FF301625FF301625A801A701272D850137
:100AC0008101C701BE01AC01AB01AA01AD01A701C3
:100AD000A801B101A201A301A40107309900831666
:100AE000031382308100811395019516151670301D
:100AF0008F04910183120313AE018B168B17FF3005
:100B0000C900CA00CB00CC00CD00CE00FF301625B6
:100B1000FF301625C901CA01CB01CC01CD01CE01A0
:100B2000FF301625FF30162552242E08CA00FF304C
:100B30001625FF3016252E1C642C5624272D41081F
:100B40008A007908420703188A0A82000A08C50049
:100B50005C088A005D088200093479340A340C3458
:100B60000A34C9340B3414340B34A7340C343A34FB
:100B700021340034213409342134183421343F34F1
:100B80002134663421347B34213496342134A53425
:100B90002134B4342134CF3404308A001324C90002
:100BA0001324CA0005308A001F304905DE001F30BB
:100BB0005E02031DE72DC901CA01CB01CC01CD01A5
:100BC000CE0105308A00162505308A00022EC91B89
:100BD000EB2D0326EC2D1726491BF02D2B26F12D8E
:100BE0003F26C91AF52D5326F62D672603308A00B5
:100BF0005708E52305308A002E18022E3118022EE0
:100C0000DE0BE72D08000D30DF00AC30840000085B
:100C1000840A800084038403DF0B072E840A80018A
:100C200040304A1B8007A030CA1B800708000D30E7
:100C3000DF00A1308400000884038000840A840A55
:100C4000DF0B1B2E8403800140304A1B8007A0303D
:100C5000CA1B800708000D30DF00BA30840000088E
:100C6000840A800084038403DF0B2F2E840A800112
:100C700040304A1A8007A030CA1A800708000D3099
:100C8000DF00AF308400000884038000840A840AF7
:100C9000DF0B432E8403800140304A1A8007A030C6
:100CA000CA1A800708000D30DF00C8308400000831
:100CB000840A800084038403DF0B572E840A80019A
:100CC00040304A198007A030CA19800708000D304B
:100CD000DF00BD308400000884038000840A840A99
:100CE000DF0B6B2E8403800140304A198007A0304F
:100CF000CA1980070800A6308400FF304A1B800014
:100D0000AC308400FF30491A8000AA308400FF30E4
:100D100049198000AE308400FF304C188000B0309C
:100D20008400FF304C198000B3308400FF30CC1AAF
:100D30008000C9308400FF30CD1A8000C7308400A5
:100D4000FF30CD198000AF308400FF30CC18800018
:100D5000A2308400FF304A198000B2308400FF3096
:100D60004C1A8000C6308400FF304D198000BC3022
:100D70008400FF304E188000BF308400FF30CE1951
:100D80008000C0308400FF304E1A8000A130840003
:100D9000FF30CA188000BE308400FF304E1980003A
:100DA000C1308400FF30CE1A8000B1308400FF30A3
:100DB000CC198000A4308400FF304A1A8000A5308E
:100DC0008400FF30CA1A8000A8308400FF30491820
:100DD0008000C5308400FF30CD188000C43084000E
:100DE000FF304D188000A9308400FF30C918800002
:100DF000B6308400FF304B188000B7308400FF30DD
:100E0000CB188000C3308400FF30CE1B8000C2307E
:100E10008400FF304E1B8000A7308400FF30CA1BC7
:100E20008000B4308400FF304C1B8000B53084005B
:100E3000FF30CC1B8000C8308400FF304D1A80008A
:100E4000AD308400FF30C91A8000BA308400FF3012
:100E50004B1A8000BB308400FF30CB1A8000AB30CF
:100E60008400FF30C9198000B8308400FF304B196E
:100E70008000B9308400FF30CB198000BD30840081
:100E8000FF30CE188000A0308400FF304A18800068
:100E9000A3308400FF30CA1980000800A03084000D
:100EA0004A18800A50188003A1308400CA18800AAA
:100EB000D0188003A23084004A19800A5019800398
:100EC000A3308400CA19800AD0198003A43084009A
:100ED0004A1A800A501A8003A5308400CA1A800A70
:100EE000D01A8003A63084004A1B800A501B80035E
:100EF000A7308400CA1B800AD01B8003A83084005E
:100F00004918800A4F188003A9308400C918800A44
:100F1000CF188003AA3084004919800A4F19800332
:100F2000AB308400C919800ACF198003AC3084002B
:100F3000491A800A4F1A8003AD308400C91A800A0A
:100F4000CF1A8003AE3084004C18800A52188003F8
:100F5000AF308400CC18800AD2188003B0308400EF
:100F60004C19800A52198003B1308400CC19800AD0
:100F7000D2198003B23084004C1A800A521A8003BE
:100F8000B3308400CC1A800AD21A8003B4308400B3
:100F90004C1B800A521B8003B5308400CC1B800A96
:100FA000D21B8003B63084004B18800A511880038E
:100FB000B7308400CB18800AD1188003B830840081
:100FC0004B19800A51198003B9308400CB19800A6B
:100FD000D1198003BA3084004B1A800A511A800359
:100FE000BB308400CB1A800AD11A8003BC30840045
:100FF0004E18800A54188003BD308400CE18800A31
:10100000D4188003BE3084004E19800A541980031E
:10101000BF308400CE19800AD4198003C030840008
:101020004E1A800A541A8003C1308400CE1A800AF6
:10103000D41A8003C23084004E1B800A541B8003E4
:10104000C3308400CE1B800AD41B8003C4308400CC
:101050004D18800A53188003C5308400CD18800ACB
:10106000D3188003C63084004D19800A53198003B9
:10107000C7308400CD19800AD3198003C83084009A
:101080004D1A800A531A8003C9308400CD1A800A91
:10109000D31A8003080004308A001324C9001324E3
:1010A000CA001324CB001324CC001324CD00132436
:1010B000CE0008308A00DA01C91B5A14491BDA1421
:1010C000CB1B5A154B1BDA15CD1B5A164D1BDA16C6
:1010D000A03084004A1871214A1C7521A130840077
:1010E000CA187121CA1C7521A23084004A197121C5
:1010F0004A1D7521A3308400CA197121CA1D7521AA
:10110000A43084004A1A71214A1E7521A53084003A
:10111000CA1A7121CA1E7521A63084004A1B71218A
:101120004A1F7521A7308400CA1B7121CA1F75216F
:10113000A830840049187121491C7521A930840008
:10114000C9187121C91C7521AA308400491971215F
:10115000491D7521AB308400C9197121C91D752144
:10116000AC308400491A7121491E7521AD308400CC
:10117000C91A7121C91E7521AE3084004C18712125
:101180004C1C7521AF308400CC187121CC1C75210A
:10119000B03084004C1971214C1D7521B130840090
:1011A000CC197121CC1D7521B23084004C1A7121EB
:1011B0004C1E7521B3308400CC1A7121CC1E7521D0
:1011C000B43084004C1B71214C1F7521B530840054
:1011D000CC1B7121CC1F7521B63084004B187121B6
:1011E0004B1C7521B7308400CB187121CB1C7521A5
:1011F000B83084004B1971214B1D7521B930840022
:10120000CB197121CB1D7521BA3084004B1A712185
:101210004B1E7521BB308400CB1A7121CB1E75216A
:10122000BC3084004E1871214E1C7521BD308400E5
:10123000CE187121CE1C7521BE3084004E1971214B
:101240004E1D7521BF308400CE197121CE1D752130
:10125000C03084004E1A71214E1E7521C1308400A9
:10126000CE1A7121CE1E7521C23084004E1B712111
:101270004E1F7521C3308400CE1B7121CE1F7521F6
:10128000C43084004D1871214D1C7521C530840077
:10129000CD187121CD1C7521C63084004D197121E6
:1012A0004D1D7521C7308400CD197121CD1D7521CB
:1012B000C83084004D1A71214D1E7521C93084003B
:1012C000CD1A7121CD1E752103308A005708E52300
:1012D00008308A002E18702931187029DA0B682816
:1012E0000800800A0319800908008008031D800394
:1012F0000800123404341834FF34FF34C03400348E
:10130000C0340034FF34FF34C0340034C0340034FF
:10131000FF34FF34C0340034C0340034FF34FF34B1
:10132000C0340034C0340034C0340034C03400341D
:10133000C0340034C0340034C0340034C03400340D
:10134000C0340034C0340034C0340034C0340034FD
:10135000C0340034C0340034C0340034FF34FF34AF
:10136000C0340034C0340034FF34FF34C03400349F
:10137000C0340034FF34FF34C0340034C03400348F
:10138000FF34FF34C0340034C0340034C03400347F
:10139000C0340034C0340034C0340034C0340034AD
:1013A000C0340034C0340034C0340034C03400349D
:1013B000C0340034C0340034C0340034C03400348D
:1013C000FF34FF34C0340034C0340034FF34FF3401
:1013D000C0340034C0340034FF34FF34C03400342F
:1013E000C0340034FF34FF34C0340034C03400341F
:1013F000C0340034C0340034C0340034C03400344D
:10140000C0340034C0340034C0340034C03400343C
:10141000C0340034C03400340F3430341F3430341E
:1014200000340034003400340034C034003400345C
:101430000034003400340C34003400340034003400
:101440000034C03400340034003400340034033439
:1014500000340034003400340034C034003400342C
:101460000034003400340034C0340034003400341C
:101470000034C0340034003400340034003400340C
:1014800030340034003400340034C03400340034CC
:1014900000340034003400340C34003400340034A0
:1014A0000034C034003400340034003400340034DC
:1014B00003340034003400340034C03400340034C9
:1014C000003400340034C0340034003400340034BC
:1014D0000034003400340034003430340034C0347C
:1014E000003400340034003400340034003400345C
:1014F00000340C340034C034003400340034003480
:101500000034003400340034003403340034C03478
:10151000003400340034003400340034003400342B
:1015200000340034C034C03400340034003400349B
:101530000034003400340034003400343034C0341B
:1015400000340034003400340034003400340034FB
:10155000003400340C34C03400340034003400341F
:101560000034003400340034003400340334C03418
:1015700000340034003400340034C034003400340B
:10158000003400340034C0340034003400340034FB
:101590000034123404340C34FF34FF34C0340034CB
:1015A000C0340034FF34FF34C0340034C03400345D
:1015B000FF34FF34C0340034C0340034FF34FF340F
:1015C000C0340034C0340034C0340034FF34FF343D
:1015D000C0340034C0340034FF34FF34C03400342D
:1015E000C0340034FF34FF34C0340034C03400341D
:1015F000FF34FF34C0340034C0340034C03400340D
:10160000FF34FF34C0340034C0340034FF34FF34BE
:10161000C0340034C0340034FF34FF34C0340034EC
:10162000C0340034FF34FF34123404341834FC3432
:101630000034FF34FC34C0347F34F8340034FF34D9
:10164000F834C034FF34F0340134FF34F034C134A2
:10165000FF34E0340334FF34E034C334FF34C034A7
:101660000734FF34C034C734FF34C0340F34FF3480
:101670008034CF34FF34C0341F34FF340034DF34BF
:10168000FF34C0343F34FE340034FF34FE34C03401
:101690007F34FC340034FF34FC34C034FF34F8347D
:1016A0000034FF34F834C134FF34F0340134FF34F3
:1016B000F034C334FF34E0340334FF34E034C7344F
:1016C000FF34C0340734FF34C034CF34FF34C03467
:1016D0000F34FF348034DF34FF34C0341F34FF3420
:1016E0000034FF34FE34C0343F34FE340034FF3461
:1016F000FC34C0347F34FC340034FF34F834C0345C
:10170000FF34F8340034FF34F034C134FF34F034A3
:101710000134FF34E034C334FF34E0340334FF34A5
:10172000C034C734FF34C0340734FF348034CF347E
:10173000FF34C0340F34FF340034DF34FF34C0349E
:101740001F34FE340034FF34FE34C0343F341234CE
:1017500004341834C0340034FF34FC34C0347F34D3
:10176000C0340034FF34F834C034FF34C0340034A3
:10177000FF34F034C134FF34C0340034FF34E0347B
:10178000C334FF34C0340034FF34C034C734FF34B2
:10179000C0340034FF348034CF34FF34C0340034DC
:1017A000FF340034DF34FF34C0340034FE340034FE
:1017B000FF34FE34C0340034FC340034FF34FC34D5
:1017C000C0340034F8340034FF34F834C03400340A
:1017D000F0340134FF34F034C0340034E0340334E6
:1017E000FF34E034C0340034C0340734FF34C03434
:1017F000C0340034C0340F34FF348034C03400347B
:10180000C0341F34FF340034C0340034C0343F349B
:10181000FE340034C0340034C0347F34FC3400342F
:10182000C0340034C034FF34F8340034C0340034E1
:10183000C134FF34F0340134C0340034C334FF34D5
:10184000E0340334C0340034C734FF34C0340734C8
:10185000C0340034CF34FF34C0340F34C0340034CB
:10186000DF34FF34C0341F34C0340034FF34FE345E
:10187000C0343F34123401343334E0340034C034E3
:101880000034C0340034F0340034C0340034C03488
:101890000034F8340034C0340034C0340034FC3434
:1018A0000034C0340034C0340034DE340034C0347A
:1018B0000034C0340034CF340034C0340034C03479
:1018C0000034C7348034C0340034C0340034C334EE
:1018D000C034C0340034C0340034C134E034C034C7
:1018E0000034C0340034C034F034C0340034C03468
:1018F0000034C0347834C0340034C0340034C034D0
:101900003C34C0340034C0340034C0341E34C034DD
:101910000034C0340034C0340F34C0340034C03418
:101920000034C0340734C0340034C0340034C03410
:101930000334C0340034C0340034C0340134C03403
:101940000034C0340034C0340034E0340034C034D7
:101950000034C0340034F0340034C0340034C034B7
:101960000034F8340034C0340034C0340034FC3463
:101970000034C0340034C0340034DE340034C034A9
:101980000034C0340034CF340034C0340034C034A8
:101990000034C7348034C0340034C0340034C3341D
:1019A000C034C0340034C0340034C134E034C034F6
:1019B0000034C0340034C034F034C0340034C03497
:1019C0000034C0347834C0340034C0340034C034FF
:1019D0003C34C0340034C0340034C0341E34C0340D
:1019E0000034C0340034C0340F34C0340034C03448
:1019F0000034C0340734C0340034C0340034C03440
:101A00000334C0340034C0340034C0340134C03432
:101A10000034C0340034C0340034E0340034C03406
:101A20000034C0340034F0340034C0340034C034E6
:101A30000034F8340034C0340034C0340034FC3492
:101A40000034C0340034C0340034DE340034C034D8
:101A50000034C0340034CF340034C0340034C034D7
:101A60000034C7348034C0340034C0340034C3344C
:101A7000C034C0340034C0340034C134E034C03425
:101A80000034C0340034C034F034C0340034C034C6
:101A90000034C0347834C0340034C0340034C0342E
:101AA0003C34C0340034C0340034C0341E34C0343C
:101AB0000034C0340034C0340F34C0340034C03477
:101AC0000034C0340734C0340034C0340034C0346F
:0E1AD0000334C0340034C0340034C034013458
:02400E00C430BC
:104200001000FF0003001F3400340134FC340D346F
:1042100000341000500006000134C0340134003472
:10422000013430340134003401340C3408340034A7
:104230001000500012008E3440340E3480348E341E
:10424000C0340E3480348E3440340E3400342E3476
:1042500004340E3408342E340C340E3408342E3426
:1042600004340E3400344E3410340E3420344E34C2
:1042700030340E3420344E3410340E3400341000F8
:10428000500012004E3450348E34A0344E34F0348A
:104290008E34A0344E3450348E3400342E344434B2
:1042A0008E3488342E34CC348E3488342E344434D6
:1042B0008E3400344E3414342E3428344E343C348E
:1042C0002E3428344E3414342E3400340F00300091
:1042D00003003F34FF340034013400340034003430
:1042E00000343F34FF3400340034003400340034F0
:1042F00000343F34FF340F00FF000400FF34FF346C
:104300000034013400340034C03400343F34FF340E
:1043100000340034C0340034003400343F34FF34FF
:10432000C034003400340034003400341000800005
:1043300006008134C0348D340034413430344D347F
:10434000003421340C342D340034100010000600E9
:104350008234C0348E340034423430344E3400342D
:1043600022340C342E3400341000FF000C001F34B3
:1043700000348F34C0341F3400340F34C0341F3441
:1043800000344F3430341F3400340F3430341F3491
:1043900000342F340C341F3400340F340C3410002C
:1043A000600006008134C0348E340034413430342F
:0E43B0004E34003421340C342E3400340034EA
:00000001FF
